:03000000022B1AB6
:0C2B1A0078FFE4F6D8FD75814B022B61BA
:100ED20020000A3C2E2E2E3E004950436F6E6E6556
:100EE20063745245510A004950436F6E6E656374D4
:100EF200000A49504E6F41434B210A003E432C5693
:100F02002C43432CC0E4E0EFF2E5F020D1E8EDEA17
:100F1200EEEC49500A003E432C4D41432C25303221
:100F220062583A25303262583A25303262583A25B0
:100F3200303262583A25303262583A25303262589D
:100F42002C4D414320E0E4F0E5F10A003E432C56EB
:100F520045522C20332E3220EEF2202573202573A9
:100F62002CC2E5F0F1E8FF20495020ECEEE4F3EB6F
:100F7200FF0A004A756E2032352032303039003196
:100F8200333A32393A3232003E432C4C442C5052DE
:100F92004F473A20202020202020202020202020DF
:100FA200202020202020202020202020202020203F
:100FB200202020202020202020202020202020202F
:100FC200202020202020202020202020202020201F
:100FD20020202020202020202CC4E0F2E020EFF06E
:100FE200EEF8E8E2EAE828F4E0E9EB290A003E2A12
:100FF2002C312CCEF1EDEEE2EDFBE520EFE0F0E05E
:10100200ECE5F2F0FB20F1E5F2E5E2EEE3EE20E8BA
:10101200EDF2E5F0F4E5E9F1E00A003E412C413061
:10102200312C2562752E2562752E2562752E25625C
:10103200752C495020E0E4F0E5F120E0E4E0EFF225
:10104200E5F0E00A003E412C4130322C2562752E3B
:101052002562752E2562752E2562752C495020E079
:10106200E4F0E5F120EEF1ED2E20F1E5F0E2E5F01D
:10107200E00A003E412C4130332C2562752E256258
:10108200752E2562752E2562752C495020E0E4F0FC
:10109200E5F120F0E5E72E20F1E5F0E2E5F0E00AE7
:1010A200003E412C4130342C2562752E2562752E6E
:1010B2002562752E2562752CCCE0F1EAE020F1E57F
:1010C200F2E80A003E412C4130352C2562752E256E
:1010D20062752E2562752E2562752CD8EBFEE70A05
:1010E200003E2A2C312CC4EEEF2E20EFE0F0E0EC93
:1010F200E5F2F0FB20F1E5F2E5E2EEE3EE20E8EDC9
:10110200F2E5F0F4E5E9F1E00A003E422C53303119
:101112002C2562752CC6E4E0F2FC20E7E0EFF0EE4D
:10112200F1E020F1EEE5E4E8EDE5EDE8FF20EEF296
:1011320020F1E5F0E2E5F0E00A003E422C533032C5
:101142002C2562752CCEE1ECE5ED20F120F1E5F0E5
:10115200E2E5F0EEEC20E1E5E720EAE2E8F2E0ED9C
:10116200F6E8E90A003E422C5330332C2562752CF6
:10117200CFE5F0E5E7E0EFF3F1EA20EFF0E820EF6A
:10118200EEF2E5F0E520F1E2FFE7E820F120F1E5FB
:10119200F0E2E5F0EEEC0A003E454E440A000A4455
:1011A200756D7058202020202030302030312030C2
:1011B2003220303320303420303520303620303762
:1011C2002030382030392030412030422030432036
:1011D2003044203045203046000A3A003A20000AC6
:1011E200000A44756D7044202020202030302030C9
:1011F2003120303220303320303420303520303628
:101202002030372030382030392030412030422001
:101212003043203044203045203046004572722051
:101222006B657900526420656570726F6D0A0052B9
:1012320064204D454D0A00526420436F64650A00E4
:10124200577269746520436F64650A00446562756C
:10125200674950204F4E0A00446562756749502025
:101262004F46460A00446562756755736572204FA2
:101272006E0A00446562756755736572204F464673
:101282000A0044656275674D7367204F6E0A004419
:10129200656275674D7367204F46460A00436F6E5D
:1012A200666967206C6F636B210A0057722065655F
:1012B20070726F6D0A0020536176652065657072E9
:1012C2006F6D210A00457272204D414321004C6F1F
:1012D20061643E3E002A003C4130313D003C4130D9
:1012E200323D003C4130333D003C4130343D003C16
:1012F2004130353D003C21003C5330313D003C53F0
:1013020030323D003C5330333D003C5330353D00DC
:061312003C5330363D00A3
:06337A00014800014600BD
:1033C700C28E438910E4F58B758DB8D2ABD28E22AD
:03001B00022A8A2C
:102A8A00C0E0C083C082C0D0C28E758B00758DB87D
:102A9A00201D0675A61E75A6E10546D219E54860F1
:102AAA00020548E547D3940140021547054BE54B1B
:102ABA00540F7048D225E54B543F7012D2179066D6
:102ACA008BE0600A04F0E0D394B44002D21D906611
:102ADA0086E0600204F0906104E0600214F09066FF
:102AEA008CE0D394014003E014F0301C020549E560
:102AFA004AD394644004D21D8002054AE545D39422
:102B0A000140021545D28ED0D0D082D083D0E03297
:10086900C291C290D2B5C2227D027C007F071233A9
:100879005D8F26E526646060097D017F601232F88C
:10088900D222E4FDFC7F0B12335D8F26E52630E68C
:10089900097D04E4FF12331CD2227D017C007F070D
:1008A90012335D8F26E5267008FD7FFF1232F8D2DC
:1008B90022302203126000C288C2A8C2AA75890028
:1008C900122EC890633EE0B4FA06A3E064CE607BC2
:1008D900E4F52674362526F582E43463F583E4F0DD
:1008E9000526E526B443EC90633E74FAF0A374CE72
:1008F900F0A374CCF0906344740AF0E4A3F0A30469
:10090900F0A3F090633A74FFF0A3F0A3F0E4A3F02E
:10091900906355740AF0E4F526E5262401FFE433D3
:10092900FE74362526F582E43463F583E0FD123240
:10093900D40526E526C3944340DFE4F5A775A61E32
:1009490075A6E1907FF0F0A3F080FE9063497403EF
:10095900F0A374CCF0E4906348F0122716C2B512E4
:1009690029F4C21D1230E7D222C224C2239065762F
:100979007408F09062B47424F0E4A3F090633EE04C
:100989009062B6F090633FE09062B7F0906340E008
:100999009062B8F0906341E09062B9F0906342E0F0
:1009A9009062BAF0906343E09062BBF0754701E44E
:1009B900906577F0C21EC21FC220C221202218AF43
:1009C90026FE7D03122480E4FF12289C7E0E7FD22E
:1009D900E4FBFDFC1220A290668BE060037401F039
:1009E900E4906104F0F549906575F0F54A1233C752
:1009F90075A70775A61E75A6E1D2AFE4F54A906101
:100A090004E070031233B090668CE06401701D90AD
:100A190080007410F09080A874FFF0A3F0A3F0A3F5
:100A2900F0E490668CF0D222C223C224908008E0C0
:100A3900F52630E405D21E7410F0E52630E508D21B
:100A4900209080087420F0E52630E608D21F9080B7
:100A5900087440F0E549C394034019908002E4F01A
:100A6900908001F0908000F0E54994064006E4F595
:100A7900491230E79080A0E07003122FC09080B82F
:100A8900E07003122F469080D0E0700312308B90F3
:100A99008000E07013301E101221A9906331EFF02D
:100AA900D394004003120026908002E070069080E3
:100AB90000E06005D21C020A04C21CE4F5499061F9
:100AC90004E06003020A04202212906578E0600CB9
:100AD9007E0E7FD4122398E4906578F030201212AC
:100AE9001DF9906331EFF0D394004005E0FF123413
:100AF90004201F03020C7A121C72906331EFF0700C
:100B090003020A04906375E054BF247F7003020B4B
:100B1900E3147003020BBB24026003020C1C2022A5
:100B2900077E0E7FDB122398202603020C7A90633E
:100B39004DE07006906351E06067906682E0FF9037
:100B4900634DE0B50724906683E0FE90634EE0B5FF
:100B59000618906684E0FE90634FE0B5060C906637
:100B690085E0FE906350E06E6037906351E06F60FE
:100B790003020C7A906683E0FF906352E06F600392
:100B8900020C7A906684E0FF906353E06F60030281
:100B99000C7A906685E0FF906354E06F6003020C65
:100BA9007AC21A9065777401F012001E7547010226
:100BB9000C7A90668BE060037401F090667AE0FF2E
:100BC900906377E06F6003020C7A90667AE004F034
:100BD900E4F547906575F0020C7A301A03020C7A35
:100BE900906344E07003020A04906355740AF0129A
:100BF90033FAD21AE4F547906575F090668604F0E9
:100C0900E4906679F0A3F02022677E0E7FE9122333
:100C190098805E90668BE060037401F0301A529000
:100C29006375E020E74B906377E0FF906679E0FE1B
:100C39006F600D906681E07007EE146F703380135A
:100C4900906679E004F0906331E0FFD394044003A7
:100C590012324F9060007482F0A37401F0906377B0
:100C6900E0906002F07E607F007D03122C2D020A65
:100C790004201A03020D92E5477068121F6AEF609B
:100C8900237E647F75906476E02404FD122C2D90F8
:100C99006681E07009906355E0F547020A04E4F5BE
:100CA90047020A04906686E0D3943C4036906681F8
:100CB900E0703090668604F01227E0E4906475F0E5
:100CC900A37412F090667AE0906477F0A374FDF053
:100CD90090610563A20190647963A2017F121219E0
:100CE900C0809E1233D78F26E526B4011590600087
:100CF9007483F0E4A3F07E607F007D02122C2D0244
:100D09000A04E526D39401401C9060007483F0A383
:100D19007401F0E52624FEA3F07E607F007D0312B6
:100D29002C2D020A04E54764016003020A04906558
:100D390075E004F02022077E0E7FF312239890635A
:100D490055E0C394C85004E02432F0906575E0C3BF
:100D59009405400DC21AE4906577F012001E020A4C
:100D6900047C667D82906349E0FAA3E0FB7F02126E
:100D79002E447E647F75906476E02404FD122C2D48
:100D8900906355E0F547020A04E5476401600302F0
:100D99000A04906577E014604624FE6042147003EB
:100DA900020E8524046003020A04E4F5492026138F
:100DB9009065777404F0906575E05401F07547010A
:100DC900020A049080027410F0E4906577F090654F
:100DD9007504F07547FA90668274FFF0020A049070
:100DE9006682E07003020E6F9064757480F09064FF
:100DF900777401F0E4A3F0A304F0A37430F0A374B2
:100E09007BF0E4F526747C2526F582E43464F583C9
:100E1900747DF0747D2526F582E43464F583E4F06D
:100E2900E5262407906476F07C667D82906349E02C
:100E3900FAA3E0FB7F02122E447E647F75E5262427
:100E490009FD122C2D906681E0601B1233FAD21A2B
:100E5900E4F547906575F090668604F0E49066794C
:100E6900F0A3F0020A04302607E4906577F08006C3
:100E79009065777404F07547FA020A049080027449
:100E890010F0754705906575E06401FFF09065778E
:100E99007401F0EF7019906351E06013FCA3E0FD59
:100EA900A3E0FEA3E0FF9066821217A7020A04904E
:100EB900634DE0FCA3E0FDA3E0FEA3E0FF906682A2
:080EC9001217A7020A0480FEC3
:010ED10022FE
:10002600906376E0B444047F0180027F009063759C
:10003600E0B447047E0180027E00EE5F604A906372
:100046003EE0906377F090633FE0906378F09063D2
:1000560040E0906379F0906341E090637AF09063BA
:1000660042E090637BF0906343E090637CF09063A2
:10007600767452F09062AE63A2019080A863A201EA
:100086007F061219C002085F906331E0C3940850DE
:100096000302086890633EE0FF906377E06F6003B9
:1000A60002086890633FE0FF906378E06F600302A8
:1000B6000868906340E0FF906379E06F6003020890
:1000C60068906341E0FF90637AE06F60030208681E
:1000D600906342E0FF90637BE06F600302086890E4
:1000E6006343E0FF90637CE06F60030208689063FF
:1000F60076E06444701A9080A8E0B4FF139062AE74
:1001060063A2019080A863A2017F061219C0801025
:100116009062B2E09080ACF09062B3E09080ADF077
:1001260090668BE060037401F090668C7464F090C6
:1001360063767452F0906375E0646D600302026941
:100146007BFF7A0E79FE12137A7BFF7A0F7918906D
:10015600633EE0F52FA3E0F530A3E0F531A3E0F52B
:1001660032A3E0F533A3E0F53412137A752FFF7549
:10017600300F7531757532FF75330F7534817BFF1E
:100186007A0F794E12137A7BFF7A0F798A12137AD5
:100196007BFF7A0F79F012137A7BFF7A10791D9024
:1001A6006344E0F52FA3E0F530A3E0F531A3E0F5D5
:1001B6003212137A7BFF7A10794790634DE0F52F60
:1001C600A3E0F530A3E0F531A3E0F53212137A7B14
:1001D600FF7A107975906351E0F52FA3E0F530A30F
:1001E600E0F531A3E0F53212137A7BFF7A1079A39A
:1001F60090633AE0F52FA3E0F530A3E0F531A3E0F4
:10020600F53212137A7BFF7A1079C6906336E0F5E1
:100216002FA3E0F530A3E0F531A3E0F53212137A0F
:100226007BFF7A1079E312137A7BFF7A11790CA29D
:1002360026E433F52F12137A7BFF7A11793C906608
:1002460081E0F52F12137A7BFF7A11796790668B1E
:10025600E0F52F12137A1232827BFF7A11799A1205
:10026600137A22906375E0644C70737E117FA0FB55
:10027600FDFC1220A290637DE0F527A3E0F528E4BB
:10028600F52AE52790637FF0A3E528F07E117FDB52
:100296007C637D7F7B021220A2E4F5298528828576
:1002A6002783E0FF747F2529F582E43463F583EF25
:1002B600F00528E528700205270529E529B410DC94
:1002C6007E117FDE7C637D7F7B101220A2052AE5EE
:1002D6002AC3941040AC7E117FE1122398229063CA
:1002E60075E0646C7060F52B7E117FE3FBFDFC12FC
:1002F60020A2E4F52AE490637FF0A3E52BF07E11BB
:100306007FDB7C637D7F7B021220A2E4F529A82B8C
:10031600E6FF747F2529F582E43463F583EFF00563
:100326002B0529E529B410E67E117FDE7C637D7FEF
:100336007B101220A2052AE52AC3940840B77E1135
:100346007FE112239822906375E0644B7061F52972
:1003560074672529F582E43463F583E060327467B7
:100366002529F582E43463F583E0F4602374672578
:1003760029F582E43463F583E0FF747D2529F5824F
:10038600E43463F583E0B507100529E529B408C010
:100396009061047432F002085F9063757421F03046
:1003A600220302085F7E127F1E12239802085F90C6
:1003B6006375E0B4521A2022077E127F2612239814
:1003C6009063757472F07E637F757D08122BA6228A
:1003D600906375E0644970452022077E127F3112D2
:1003E600239890637DE0F527A3E0F528E4F52985B9
:1003F6002882852783E0FF747F2529F582E434630C
:10040600F583EFF00528E528700205270529E5297B
:10041600B480DC7E637F757D8A122BA6229063757D
:10042600E0644370462022077E127F39122398909B
:10043600637DE0F527A3E0F528E4F5298528828584
:100446002783E493FF747F2529F582E43463F583DB
:10045600EFF00528E528700205270529E529B4806F
:10046600DB7E637F757D8A122BA622906375E0641E
:100476005A70532022077E127F4212239890637D82
:10048600E0F527A3E0F5287C637D7F7B80AF28AE6F
:100496002712321BE4F529852882852783E493FFFA
:1004A600747F2529F582E43463F583EFF00528E5AA
:1004B60028700205270529E529B480DB7E637F7550
:1004C6007D8A122BA622906375E0644460030205C0
:1004D6005D90637DE0FF6444700302085FEFB43112
:1004E6000CC2227E127F4E12239802085F90637D13
:1004F600E0B4300CD2227E127F5A12239802085F93
:1005060090637DE0B4320CD2237E127F671223986B
:1005160002085F90637DE0B4330CC2237E127F75C0
:1005260012239802085F90637DE0B4340CD2247ED7
:10053600127F8412239802085F90637DE0B4350C25
:10054600C2247E127F9112239802085F90637DE099
:10055600FF12340302085F906104E0701320220743
:100566007E127F9F1223989063757421F002085FB4
:100576009061047432F0906375E0FFB45104C2AF29
:1005860080FEEF645770452022077E127FAD12234E
:100596009890637EE0906331F0E4F529906331E052
:1005A600FFE529C39F400302085F747F2529F58272
:1005B600E43463F583E0FF90637DE0252924ADF5FF
:1005C60082E43461F583EFF0052980D0906375E00D
:1005D600645360030206802022077E127FB812232E
:1005E6009890633EE0FF9061B6E06F703C90633F89
:1005F600E0FF9061B7E06F7030906340E0FF90617C
:10060600B8E0B50724906341E0FF9061B9E0B50713
:1006160018906342E0FF9061BAE0B5070C9063431F
:10062600E0FF9061BBE06F60169063757421F03057
:10063600220302085F7E127FC712239802085FE436
:10064600F529E4F54AAF29FE74AD2529F582E4348F
:1006560061F583E0FD1232D40529E529C394FE40F5
:10066600E1C2AFE4907FF0F0A3F0907FFD74AAF0B2
:10067600A374FFF0A37455F080FE906375E0644F99
:10068600704C90637DE0F527A3E0F528E528452723
:10069600700A2022077E127FD01223982022077E1E
:1006A600127FD7122398E4F529747F2529F582E471
:1006B6003463F583E0852882852783F00528E528BD
:1006C600700205270529E529B480DE02085F9063DC
:1006D60075E0FFB4452190637DE0FDA3E0907FF0D7
:1006E600CDF0A3EDF0C2AF907FFD74AAF0A374FF26
:1006F600F0A37455F080FEEF64656003020868900D
:10070600637DE0FFA3E0907FF0CFF0A3EFF0E4F588
:1007160027F528D3907FF1E09528907FF0E0952784
:100726004020E4F54A2528FFE5273401FE85288286
:10073600852783E0FD1232D40528E52870020527B7
:1007460080D17E127FD9122D3AEF4E60201200031F
:10075600906344EFF0120003906345EFF01200033C
:10076600906346EFF0120003906347EFF07E127F2E
:10077600DF122D3AEF4E602012000390634DEFF02A
:1007860012000390634EEFF012000390634FEFF0F8
:10079600120003906350EFF07E127FE5122D3AEFC0
:1007A6004E6020120003906351EFF0120003906335
:1007B60052EFF0120003906353EFF01200039063C0
:1007C60054EFF07E127FEB122D3AEF4E60201200AE
:1007D6000390633AEFF012000390633BEFF01200D0
:1007E6000390633CEFF012000390633DEFF07E123E
:1007F6007FF1122D3AEF4E6020120003906336EF20
:10080600F0120003906337EFF0120003906338EFA5
:10081600F0120003906339EFF0E4F529E4F54AE5B8
:10082600292401FFE433FE74362529F582E4346376
:10083600F583E0FD1232D40529E529C3944340DC53
:10084600C2AFE4907FF0F0A3F0907FFD74AAF0A30E
:1008560074FFF0A37455F080FE7E637F757D0812E9
:020866002BA6BF
:01086800226D
:1031E300AE07EEC39430400BEED394395005EE2472
:1031F300D0FF22EEC39461400BEED394665005EEEC
:1032030024A9FF22EEC39441400BEED3944650050C
:08321300EE24C9FF22AF0622E0
:103396009062ADE004F070069062ACE004F09062DA
:0A33A600ACE0FEA3E0FF123340226A
:100003001233961231E3EFC454F0FEC00612339656
:080013001231E3D0E02FFF22BF
:10302E00E49069BFF01233969069C0EFF0C394300C
:10303E004018E0FFD3943950119069BFE02405F594
:10304E0082E43461F583EFF080119069BFE02405CE
:10305E00F582E43461F583E4F0800C9069BFE004FE
:10306E00F0E0D3940840BE7532007533007534001D
:0C307E00E4F5357B017A617905121ACE69
:01308A002223
:042D3A008E2C8F2D1F
:102D3E009062ACE4F0A374FFF0123396EF606EF481
:102D4E00606B852D82852C83E493B507EC752E017F
:102D5E00E52D252EF582E4352CF583E49360259040
:102D6E0062ADE0252EFF9062ACE03400FE123340DF
:102D7E00E52D252EF582E4352CF583E493B5070475
:102D8E00052E80CCE52D252EF582E4352CF583E439
:102D9E009370A6E52E24FFFFE434FFFE9062ADE0B3
:102DAE002FF09062ACE03EF07E007F0122E4FEFF49
:012DBE0022F2
:102716007E127FF7122D3AEF4E70037F01227E1252
:102726007FFA122D3AEF4E600C123396EF24D02426
:10273600FF92268002D2267E137F00122D3AEF4E9C
:10274600600C123396EF24D0906681F08005E490F9
:102756006681F07E137F06122D3AEF4E600C12331F
:1027660096EF24D090668BF08005E490668BF07E21
:10277600137F0C122D3AEF4E600C123396EF24D0D5
:1027860024FF92188002C21890633E63A2019066ED
:102796007B63A2017F061219C030183B7E137F129D
:1027A600122D3AEF4E603012000390667BEFF01266
:1027B600000390667CEFF012000390667DEFF01246
:1027C600000390667EEFF012000390667FEFF01232
:0A27D6000003906680EFF07F002200
:10319A00906576E0C3947C40027F0A906576E0FEF3
:1031AA0004F074B42EF582E43462F583EFF0BF0ABA
:1031BA0027906576E0FF04F074B42FF582E4346258
:1031CA00F583E4F0906576E0FF122DBF9065767482
:0931DA0008F09062B5E004F02257
:1030E7009080007480F090633663A201F583F582C7
:1030F70063A2017F081219C090633E63A20190800A
:103107008863A2017F0A1219C09080927407F0A306
:1031170074D0F0A37406F0906348E0FF9080B1F09C
:103127009080E1EFF09080957455F0A3F0908000C7
:0A3137007401F090800974F0F0229A
:102FC000908009E04410F09080A0E070609080A1B3
:102FD0007482F09080A874FFF0A3F0A3F0A3F07FB8
:102FE000039080AEEFF0A374CBF09080007402F0F9
:102FF0009069B31217B3000000009069B3E09080AD
:1030000040F09069B4E0908041F09069B5E0908024
:1030100042F09069B6E0908043F0A3E4F0A3F0A3FF
:0D302000F0A3F0908018F0A3F0A3F0A3F04F
:01302D002280
:10308B00908009E04440F09080D17482F07F0390EF
:10309B0080DEEFF0A374CCF09080027402F09069A4
:1030AB00B71217B3000000009069B7E0908058F09A
:1030BB009069B8E0908059F09069B9E090805AF02F
:1030CB009069BAE090805BF0A3E4F0A3F0A3F0A3C7
:0B30DB00F0908030F0A3F0A3F0A3F011
:0130E60022C7
:102F4600908009E04420F09080B8E0706C9080B9E1
:102F56007482F07F039080C6EFF07FCDA3EFF07F01
:102F6600039080C4EFF0A374CDF09080C074FFF09E
:102F7600A3F0A3F0A3F09080017402F09069BB1255
:102F860017B3000000009069BBE090804CF0906998
:102F9600BCE090804DF09069BDE090804EF0906965
:102FA600BEE090804FF0A3E4F0A3F0A3F0A3F0906E
:092FB6008024F0A3F0A3F0A3F0C5
:012FBF0022EF
:102E44008C278D28A907EAFDE975F018A424ACFFA6
:102E5400E5F034808F82F583EDF0EBFDE975F01831
:102E6400A4FFAEF024ACFBEE34808B82F583A3ED9B
:102E7400F08528828C83E0FDEF24A8FFEE3480FEE9
:102E84008F82F583EDF08528828C83A3E08F828E78
:102E940083A3F0852882852783A3A3E0FDE975F049
:102EA40018A424A8FFE5F03480FE8F82F583A3A341
:102EB400EDF08528828C83A3A3A3E08F828E83A365
:042EC400A3A3F022B2
:062BA6008D2CAB07AA060E
:102BAC00908000E030E5079065787401F022906920
:102BBC00B3E0FCA3E0FDA3E0FEA3E0F5308E2F8D87
:102BCC002E8C2DAE02AF038E838F8263A201E52F74
:102BDC00540744C0F58385308263A201AF2C121ACE
:102BEC0032E4FCFDFEE530252CF530EE352FF52FCB
:102BFC00ED352EF52EEC352DF52D908040E52DF094
:102C0C00A3E52EF0A3E52FF0A3E530F0908000743F
:102C1C0020F0AF30AE2FAD2EAC2D9069B31217A7AC
:012C2C002285
:062C2D008D27AB07AA068B
:102C3300908002E030E5079065787403F022906994
:102C4300B7E0FCA3E0FDA3E0FEA3E0F52B8E2A8D05
:102C5300298C28AE02AF038E838F8263A201E52AFB
:102C6300540744D0F583852B8263A201AF27121A40
:102C730032E4FCFDFEE52B2527F52BEE352AF52A5C
:102C8300ED3529F529EC3528F528908058E528F00D
:102C9300A3E529F0A3E52AF0A3E52BF090800274C5
:102CA30020F0AF2BAE2AAD29AC289069B71217A735
:012CB30022FE
:02289C008F2784
:10289E00908001E030E5099065787402F07F0022A7
:1028AE009069BBE0FCA3E0FDA3E0FEA3E0F52B8E58
:1028BE002A8D298C2890667B63A201E52A54074451
:1028CE00C8F583852B8263A2017F06121A48E52B79
:1028DE002406F52BE4352AF52AE43529F529E435C5
:1028EE0028F52890657963A201E52A540744C8F5B6
:1028FE0083852B8263A201AF27121A48E4FCFDFEEA
:10290E00E52B2527F52BEE352AF52AED3529F52968
:10291E00EC3528F52890804CE528F0A3E529F0A3A6
:10292E00E52AF0A3E52BF09080017420F0AF2BAEDA
:0D293E002AAD29AC289069BB1217A7AF275E
:01294B002269
:1021A9009081E0E0F527052705270527052705275D
:1021B90005270527052705270527908010E0F52A1B
:1021C900A3E0F52BA3E0F52CA3E0F52D9081E1E048
:1021D900F5270527052705270527052705270527A6
:1021E900052705270527908014E0F52EA3E0F52F94
:1021F900A3E0F530A3E0F531E530B52C08E531B5BC
:102209002D037F0022E4F527E530540744E0F583E8
:1022190085318263A20190637563A2017F08121A56
:102229007890637763A2019062AE63A2017F061280
:1022390019C0906375E0F528A3E0F529E4F5279026
:102249006375E0702AA3E024F8F527E530540744C4
:10225900E0F58385318274082582F582E43583F5BA
:102269008363A20190637563A201AF27121A78AE46
:1022790028E4FCFDE5312529F531E5303EF530ED61
:10228900352FF52FEC352EF52E908014E52EF0A381
:10229900E52FF0A3E530F0A3E531F090800074401C
:0322A900F0AF276C
:0122AC00220F
:101C72009081E6E0F5270527052705270527052793
:101C820005270527052705270527908028E0F52A3F
:101C9200A3E0F52BA3E0F52CA3E0F52D9081E7E07E
:101CA200F5270527052705270527052705270527E2
:101CB20005270527052790802CE0F52EA3E0F52FB8
:101CC200A3E0F530A3E0F531E4F527E530B52C0AC1
:101CD200E531B52D05C21F021DDEE530540744F083
:101CE200F58385318263A20190637563A2017F0847
:101CF200121A78906375E0F528A3E0F529E52945E5
:101D02002870099080027410F07F0022906682E0B1
:101D1200FFF46030906377E06F6003021DA5906668
:101D220083E0FF906378E06F7079906684E0FF90C3
:101D32006379E06F706D906685E0FF90637AE06F83
:101D42006031805F906377E0906682F0906378E024
:101D5200906683F0906379E0906684F090637AE015
:101D6200906685F090637BE0FFA3E0906349CFF03B
:101D7200A3EFF0906375E0702AA3E024F8F527E55D
:101D820030540744F0F58385318274082582F58248
:101D9200E43583F58363A20190637563A201AF27E3
:101DA200121A78AE28E4FCFDE5312529F531E5303B
:101DB2003EF530ED352FF52FEC352EF52EAF2DAE4D
:101DC2002CAD2BAC2AAB31AA30A92FA82ED31217D7
:101DD2009640099080027410F07F002290802CE5DA
:101DE2002EF0A3E52FF0A3E530F0A3E531F09080CB
:061DF200027440F0AF276F
:011DF80022C8
:101DF9009081E3E0F527052705270527052705270E
:101E09000527052705270527052790801CE0F52AC2
:101E1900A3E0F52BA3E0F52CA3E0F52D9081E4E0F8
:101E2900F527052705270527052705270527052759
:101E3900052705270527908020E0F52EA3E0F52F3B
:101E4900A3E0F530A3E0F531E4F527E530B52C0A38
:101E5900E531B52D05C220021F4FE530540744E88E
:101E6900F58385318263A20190600463A2017F0E2C
:101E7900121A8E906004E0F528A3E0F52990600C11
:101E8900E0FFF4604A90667BE0FEEF6E7079A3E0B4
:101E9900FF90600DE06F706F90667DE0FF90600EBF
:101EA900E06F706390667EE0FF90600FE06F70579F
:101EB90090667FE0FF906010E06F704B906680E065
:101EC900FF906011E06F703FE4906013F08008901C
:101ED900601374FFF0D2D9906004E0702AA3E02463
:101EE900F2F527E530540744E8F583853182740E0D
:101EF9002582F582E43583F58363A201906004634A
:101F0900A201AF27121A8EAE28E4FCFDE53125297E
:101F1900F531E5303EF530ED352FF52FEC352EF561
:101F29002EAF2DAE2CAD2BAC2AAB31AA30A92FA8E0
:101F39002ED31217965006E529452870099080017D
:101F49007410F07F0022908020E52EF0A3E52FF099
:101F5900A3E530F0A3E531F09080017440F0AF279C
:011F69002255
:042398008E2C8F2DCB
:10239C00908000E030E5079065787401F022906938
:1023AC00B3E0FCA3E0FDA3E0FEA3E0F5338E328D99
:1023BC00318C30E533FFE5325407FEE42FF52FEE78
:1023CC0034C0F52E852F82F5837423F0052FE52F6D
:1023DC007002052E532EC7F582852E83740AF005E4
:1023EC002FE52F7002052E532EC790633E63A2017A
:1023FC00852E83852F8263A2017F06121A32740602
:10240C00252FF52FE4352EF52E852C83852D826313
:10241C00A201852E83852F8263A201121A16E4FC79
:10242C00FDFE9069B3E0F8A3E0F9A3E0FAA3E02F76
:10243C00FFEE3AFEED39FDEC38FCEF2408FFE43EEC
:10244C00FEE43DFDE43CFC9069B31217A79069B320
:10245C00E0908040F09069B4E0908041F09069B5D4
:10246C00E0908042F09069B6E0908043F09080005C
:03247C007420F0D9
:01247F00223A
:0A20A2008E2C8F2D8C2E8D2F8B308D
:1020AC00908000E030E5079065787401F02290692B
:1020BC00B3E0FCA3E0FDA3E0FEA3E0F5368E358D86
:1020CC00348C33E536FFE5355407FEE42FF532EE5C
:1020DC0034C0F531853282F5837423F00532E53254
:1020EC00700205315331C7F582853183740AF005CE
:1020FC0032E532700205315331C790633E63A20161
:10210C0085318385328263A2017F06121A327406EE
:10211C002532F532E43531F531852C83852D8263FA
:10212C00A20185318385328263A201121A168F3780
:10213C00EF2532F532E43531F531E5306017852E77
:10214C0083852F8263A20185318385328263A2014C
:10215C00AF30121A32E53724082530F530FFE4FC95
:10216C00FDFEE5362FF536EE3535F535ED3534F526
:10217C0034EC3533F533908040E533F0A3E534F09F
:10218C00A3E535F0A3E536F09080007420F0AF366F
:0C219C00AE35AD34AC339069B31217A718
:0121A8002214
:062561008E2C8F2D8D2E43
:10256700908000E030E5079065787401F02290696B
:10257700B3E0FCA3E0FDA3E0FEA3E0F5348E338DCA
:10258700328C31E534FFE5335407FEE42FF530EEA6
:1025970034C0F52F853082F5837423F00530E5309C
:1025A7007002052F532FC7F582852F83EBF0053077
:1025B700E5307002052F532FC790633E63A2018554
:1025C7002F8385308263A2017F06121A3274062593
:1025D70030F530E4352FF52F852C83852D8263A2C6
:1025E70001852F8385308263A201AF2E121A3274C0
:1025F70008252EF52EFFE4FCFDFEE5342FF534EE1D
:102607003533F533ED3532F532EC3531F531908030
:1026170040E531F0A3E532F0A3E533F0A3E534F06C
:102627009080007420F0AF34AE33AD32AC31906996
:04263700B31217A71C
:01263B00227C
:022DBF008F4043
:102DC100908000E030E5079065787401F022906909
:102DD100B3E0FCA3E0FDA3E0FEA3E0F5448E438D48
:102DE100428C41E544FFE5435407FEE42FFFEE34F6
:102DF100C09062B463A201F5838F8263A201AF40E8
:102E0100121A32E4FCFDFEE5442540F544EE35435B
:102E1100F543ED3542F542EC3541F541908040E511
:102E210041F0A3E542F0A3E543F0A3E544F090802F
:102E3100007420F0AF44AE43AD42AC419069B3128F
:022E410017A7D1
:012E4300226C
:062480008E278F28AB053A
:10248600908000E030E5079065787401F02290694D
:10249600B3E0FCA3E0FDA3E0FEA3E0F52E8E2D8DB8
:1024A6002C8C2BE52EFFE52D5407FEE42FF52AEEA6
:1024B60034C0F529852A82F5837423F0052AE52A96
:1024C600700205295329C7F582852983EBF0052A71
:1024D600E52A7002052990633E63A201852983855A
:1024E6002A8263A2017F06121A327406252AF52A69
:1024F600E43529F5295329C7E527852A82852983C5
:10250600F0052AE52A700205295329C7F58285298F
:1025160083E528F0052AE52A700205295329C7E52F
:102526002E240AF52EE4352DF52DE4352CF52CE474
:10253600352BF52B908040E52BF0A3E52CF0A3E599
:102546002DF0A3E52EF09080007420F0AF2EAE2D76
:0A255600AD2CAC2B9069B31217A74F
:012560002258
:0A33E500E4FEEEC39F50030E80F8D3
:0133EF0022BB
:10334000A2AF9227C2AF438E2075D2028F828E83A6
:0C335000E0FFE4F5D2538EDFA22792AF1D
:01335C00224E
:1032D400E5D220E0FBA2AF9227C2AF43D2028F8295
:1032E4008E83EDF075D25063D250A22792AFE5D20F
:0332F40020E0FBDC
:0132F70022B4
:102EC800E4FDED2401FFE433FE12334074362DF5A2
:102ED80082E43463F583EFF00DBD3FE6E4FDED24B5
:102EE8007FFFE433FE123340742D2DF582E4346104
:102EF800F583EFF0742D2DF582E43461F583E070ED
:102F08001B742D2DF582E43461F5837420F0742E42
:102F18002DF582E43461F583E4F080040DBD80BEB4
:102F2800E49061ACF0FDEDFF7E0012334074AD2DEE
:0D2F3800F582E43461F583EFF00DBDFEE994
:012F45002269
:02321B008B2CFA
:10321D00A2AF9227C2AF85A22D53A2FE8E838F82BD
:10322D0005A28C838D827409121ABCE52C53A2FE63
:10323D0043A220121ABE53A2DF852DA2A22792AF60
:01324D00FF81
:01324E00225D
:10335D00A2AF9227C2AF8C838D82EF121ABC43A20B
:0C336D0020121ABE53A2DFA22792AFFF6D
:013379002231
:0232F8008F271E
:1032FA00A2AF9227C2AFE4F5838D827406121ABC7C
:10330A00E52743A220121ABE53A2DFA22792AF7F5B
:01331A0001B1
:01331B00228F
:02331C008F27F9
:10331E00A2AF9227C2AFE4F5838D82740A121ABC53
:10332E00E52743A220121ABE53A2DFA22792AF7F37
:01333E00018D
:01333F00226B
:1018E500A907E7FFA805EF93C3966008403B74FC82
:1018F5002FFF80F00F08EF93C3966008402B74FB11
:101905002FFF80E00F08EF93C3966008401B74FA21
:101915002FFF80D00F08EF93D3966008400B74F922
:101925002FFF80C01F1F1F1F1FEF54FEF80303F773
:10193500E893FC08E893FD08E893FE08E893FF2286
:1019450009E993C39D6008402974FB29F980F109D1
:10195500E993C39E6008401A74FA29F980E209E9FF
:1019650093D39F6008400B74F929F980D31919198D
:101975001919E9C313C313FF22740093F8ECC39834
:101985004024701F740193F8EDC3984019701474C6
:0E1995000293F8EEC398400E7009740393F8A5
:1019A300EFC39840037F00227F0122EDF8E6F008A1
:1019B300A3DFFA22EDF8E0F608A3DFFA22E0A3633F
:1019C300A201F0A363A201DFF475A2002263A201C6
:1019D300F0A363A20122E0A363A201F0A363A20127
:1019E300E0A363A201F0A363A201E463A201F0A355
:1019F30063A201DFE175A20022E0A363A2016DFEF1
:101A0300936CFDEE058393FC158363A201DFEA75F6
:101A1300A200227F00E493A363A201F00F600CA352
:101A2300E583C2E3F58363A20180EA75A20022E0A5
:101A3300A363A201F0A3E583C2E3F58363A201DFFD
:101A4300EE75A20022E0A363A201F0A3E583C2E442
:101A5300D2E3F58363A201DFEC75A20022E0A36366
:101A6300A201F0A3E58344F8C2E5F58363A201DF95
:101A7300EC75A20022E583C2E3F583E0A363A20130
:101A8300F0A363A201DFEE75A20022E583C2E4D2D4
:0A1A9300E3F583E0A363A201F0A3D2
:101A9D0063A201DFEC75A20022E58344F8F583E033
:101AAD00A363A201F0A363A201DFEE75A20022F9E8
:101ABD0022C002C004C00612FFF0D006D004D0022E
:011ACD0022F6
:102CB4005452414E5A00000AC1F3F4E5F020E7E013
:102CC400EDFFF221000A436865636B73756D20653F
:102CD40072726F7221202000CCEEE4F3EBFC20EF43
:102CE400EEE4E4E5F0E6EAE820EEE1ECE5EDE020F0
:102CF40000F120CAD93228332920C1D3D920CAEE01
:102D0400ECEFE0F120F7E5F0E5E720E0E4E0EFF2B6
:102D1400E5F020D1CECC2DC0CCCA0A00CEEFF6E827
:102D2400E820EDE0F1F2F0EEE9EAE83A20000A00EA
:062D3400FF2CB4FF2CBAD5
:1033800052668D00000000000000000000000000F8
:05339000000000000038
:0134030022A6
:0300230002294C63
:0B294C00C0E0C083C082C0D075D0186E
:1029570030984E754801AF99200224301341EF603B
:102967003EEFD39420503874AD250EF582E43467DA
:10297700F583EFF0050ED20225E004F508802074F8
:10298700AD250EF582E43467F583EFF0050ED50823
:102997000E9067ABE50EF0630E80530E80C202C245
:1029A7009830993E300339301007309704D20080B1
:1029B7002F90669FE0FFE510C39F4011C203D2131B
:1029C700C290200B02D215C20BD2968013AF10050E
:1029D7001074AD2FF582E43468F583E0F511F599AD
:0429E700C299D2AF10
:0929EB00D0D0D082D083D0E032BC
:023141008F2FCE
:103143009067ACE0FF04F074A02FF582E43466F5D9
:10315300837420F0E4FFEFC39D503BE52F75F0032C
:10316300A42434F582E4342DF583E493FB740193B2
:10317300FA740293F98F8275830012168DFE90679D
:10318300ACE024A0F582E43466F583EEF00F90679B
:06319300ACE004F080C076
:013199002213
:1032AD00742D2FF582E43461F583E0FE6420601601
:1032BD009067ACE0FD04F074A02DF582E43466F562
:0632CD0083EEF00F80DA31
:0132D30022D8
:10263C00E4F527E52775F003A42434F582E4342D62
:10264C00F583E493FB740193FA740293F9121674F4
:10265C007003022715E4F529F52AF528742D252891
:10266C00F582E43461F583E0FF7003022710E5275F
:10267C0075F003A42434F582E4342DF583E493FB44
:10268C00740193FA740293F98529827583001216EA
:10269C008DFEEFB50607752A0105298062E52A60D3
:1026AC005EEE7056AD29AF27123141E5277055AF5C
:1026BC00281232AD742D2528F9E43461FA7B01C05F
:1026CC00031B8B32753300753400E4F535D00312DF
:1026DC001ACE8F2E8E2D8D2C8C2BAB2EAA2DA92C99
:1026EC00A82B7F007E8C7D0A7C001216F6121788B0
:1026FC009069ADEEF0A3EFF0800AE4F52AF5290518
:09270C0028022668052702263F79
:0127150022A1
:1029F400C203C215C208C202C20FE4F51090669F5A
:102A0400F0F50AF50EF548C200D297D296C209C273
:102A140012C210D20CD2139069AD74FFF0A374F4F7
:102A2400F0750CFFE49067ACF075090CC206C21493
:102A3400C205C20AC2119067AA7409F0750F05E4B1
:102A4400F50D12263CC2ADE4F5C9D2CDD2CCC2C933
:102A5400C2CAF5CDF5CC9069ADE0F5CBA3E0F5CADB
:102A640085CBCD85CACCE4F5985387BFD29E4387E6
:102A740040C29FC2ACC298C29975B81075B710D243
:062A8400CAD29CD2AC2274
:0134040022A5
:0222AD008D287A
:1022AF00E4F529F52BF52AAA06A9077B018B2E8ABF
:1022BF002F8930752C68752DAF121674FF33333399
:1022CF0054F89068AEF0252AF52A74012530F530C0
:1022DF00E4352FF52F74012530F530E4352FF52F28
:1022EF00E4FFE52824FEFEEFC39E502EAB2E0530F3
:1022FF00E530AA2F7002052F14F9121674FEEF2481
:10230F0002FDE433FCED640124ADF58274683CF505
:10231F0083EEF0252AF52A0F80C8E52804F5293029
:10232F00E0020529E529C313149068ADF0252AF5BD
:10233F002AF404FEEF2402FDE433FCED640124AD26
:10234F00F58274683CF583EEF00FEF2402FFE4335F
:10235F00FEEF640124ADF58274683EF583E4F0C2AC
:10236F0002906693E0FCA3E0FDA3E0FEA3E0FFE490
:10237F00FAF9F8EF2401FFEA3EFEE93DFDE83CFCE7
:08238F009066931217A7AF2915
:012397002223
:1027E000E4FF9067AAE0FE7D000FED2405F582E48A
:1027F0003461F583EEF00F74052401F582E4346151
:10280000F583E4F07C667D92FEED1DAA0470011C48
:10281000F5828A83E0FBAA070F74052AF582E43467
:1028200061F583EBF00EBE04E07C667D96E4FEED80
:102830001DAA0470011CF5828A83E0FBAA070F74AD
:10284000052AF582E43461F583EBF00EBE04E07CEA
:10285000667D9AE4FEED1DAA0470011CF5828A8350
:10286000E0FBAA070F74052AF582E43461F583EBD7
:10287000F00EBE04E07C667D9EE4FEED1DAA0470B1
:10288000011CF5828A83E0FBAA070F74052AF582F2
:0B289000E43461F583EBF00EBE04E0C1
:01289B00221A
:0A33F000C2992099FDD299D29022D3
:0933FA00D2CAD29CD2ACC2082256
:10324F008F273003087E2C7FBB1223982290637840
:10325F00E09067AAF07E637F79E52724FCFD1222B8
:10326F00AD90669FEFF0E4F510D203C2961233F0E3
:03327F00C2152253
:101F6A00200603300B037F00229067ABE070030268
:101F7A002097FF547FF9E4906475F0A3E9F0906626
:101F8A007AE0906477F0A37416F07527647528795F
:101F9A00E4FEEF5480FF24AEF582E43467F583E073
:101FAA002EFE131313541FFD0528E528AA277002D5
:101FBA00052714F5828A83EDF074AD2FF582E43497
:101FCA0067F583E0FF0528E528AC2770020527148A
:101FDA00F5828C83EFF02EFEE4FFE924FEFDEFC3C9
:101FEA009D502BEF2402FDE433FCED640124ADF592
:101FFA008274673CF583E0FD0528E528AA2770026C
:10200A00052714F5828A83EDF02EFE0F80CCEE6050
:10201A0050906697E0FCA3E0FDA3E0FEA3E0FFE496
:10202A00FAF9F8EF2401FFEA3EFEE93DFDE83CFC3F
:10203A009066971217A72022217E2C7FC912239817
:10204A009067ABE0FD548024ADF582E43467AF823B
:10205A00FEED547FFDE4FB122561E49067ABF0804E
:10206A002C90668FE0FCA3E0FDA3E0FEA3E0FFE472
:10207A00FAF9F8EF2401FFEA3EFEE93DFDE83CFCEF
:10208A0090668F1217A7E49067ABF0D21630160548
:07209A00C2167F01227F0046
:0120A100221C
:103282007E2C7FDC1223987E2C7FF51223987E2DD4
:103292007F201223987E667FA09067ACE0FD7B05BD
:0B32A2001225617E2D7F32122398223E
:05001E00C2AEC2AC22DD
:1033B000300008209705C2001233F0E545B401063D
:0733C000E4F5451233F02291
:0E33D700301508201405C2157F01227F002248
:102B2600020869E493A3F8E493A34003F68001F254
:102B360008DFF48029E493A3F85407240CC8C333B0
:102B4600C4540F4420C8834004F456800146F6DF7F
:102B5600E4800B010204081020408090337AE47E62
:102B6600019360BCA3FF543F30E509541FFEE49374
:102B7600A360010ECF54C025E060A840B8E493A33B
:102B8600FAE493A3F8E493A3C8C582C8CAC583CA66
:102B9600F0A3C8C582C8CAC583CADFE9DEE780BE1E
:013395000037
:10167400BB010689828A83E0225002E722BBFE0274
:09168400E32289828A83E49322A7
:10168D00BB010CE58229F582E5833AF583E0225012
:10169D0006E92582F8E622BBFE06E92582F8E2225C
:0D16AD00E58229F582E5833AF583E4932276
:1016BA0075F008758200EF2FFFEE33FECD33CDCCE7
:1016CA0033CCC58233C5829BED9AEC99E58298406A
:1016DA000CF582EE9BFEED9AFDEC99FC0FD5F0D647
:1016EA00E4CEFBE4CDFAE4CCF9A88222B800C1B971
:1016FA000059BA002DEC8BF084CFCECDFCE5F0CBAF
:10170A00F97818EF2FFFEE33FEED33FDEC33FCEBE7
:10171A0033FB10D703994004EB99FB0FD8E5E4F9A2
:10172A00FA227818EF2FFFEE33FEED33FDEC33FC8F
:10173A00C933C910D7059BE99A4007EC9BFCE99A83
:10174A00F90FD8E0E4C9FAE4CCFB2275F010EF2FC8
:10175A00FFEE33FEED33FDCC33CCC833C810D707C8
:10176A009BEC9AE899400AED9BFDEC9AFCE899F803
:0E177A000FD5F0DAE4CDFBE4CCFAE4C8F92296
:0E178800C3E49FFFE49EFEE49DFDE49CFC2272
:10179600EB9FF5F0EA9E42F0E99D42F0E89C45F0A9
:0117A6002220
:0C17A700ECF0A3EDF0A3EEF0A3EFF022B5
:1017B300A8828583F0D083D0821217CA1217CA1267
:1017C30017CA1217CAE473E493A3C583C5F0C5838C
:1017D300C8C582C8F0A3C583C5F0C583C8C582C880
:0117E30022E3
:10131800E53B242FF8E6053B22782C302E02782F67
:10132800E475F0011218450216742027EB7F2ED2BF
:10133800278018EF540F2490D43440D4FF302B0B5F
:10134800EF24BFB41A0050032461FFE53C60021586
:101358003C053FE53F7002053E302E0D782CE475C4
:10136800F001121845EF0217E402319A7403D22EE5
:101378008003E4C22EF53B8B2C8A2D892EE4F53CA4
:10138800F53EF53FE53C60077F2012135380F57565
:101398003DFFC228C227C229C22AC22CC22DC22F91
:1013A800121321FF700D302E057F00121364AF3F1A
:1013B800AE3E22B4255FC2D5C22B121321FF24D022
:1013C800B40A00501A75F00A783C30D50508B6FF03
:1013D8000106C6A426F620D5047002D22A80D92494
:1013E800CFB41A00EF5004C2E5D22B021564D228FC
:1013F80080C6D22780C0D22980BCD2D580BAD22C50
:1014080080B47F201213532029077401B53C004093
:10141800F1121318FF12135302138CD22FD22D80FE
:1014280095121318FB121318FA121318F94A4B7075
:101438000679357A167BFF20292EE53C602A7E0046
:101448008E8275830012168D60060EEE653D70F073
:10145800C2D5EBC0E0EAC0E0E9C0E0EE1215ABD0BF
:10146800E0F9D0E0FAD0E0FB121674FF60AAEBC0F6
:10147800E0EAC0E0E9C0E0121353D0E02401F9D05B
:10148800E03400FAD0E0FBE53D0460DCD53DD980CE
:10149800877BFF7A1579A7D229809C7910800279F9
:1014A80008C22DC22F8008D2D5790A8004790AC2D1
:1014B800D5E53D047002F53DE4FAFDFEFF12131870
:1014C800FC7B08202813121318FD7B1030270A1202
:1014D8001318FE121318FF7B20EC3382D592D550D7
:1014E80013C3E43027069FFFE49EFEE42028039DF3
:1014F800FDE49CFCE4CBF8C228EC700CCFCECDCC3C
:10150800E824F8F870F38017C3EF33FFEE33FEEDED
:1015180033FDEC33FCEB33FB994002FB0FD8E9EBCE
:10152800302805F8D0E0C448B228C0E00AEC4D4E97
:101538004F78207B0070C2EAB53D0040BCC0E01285
:1015480015ADD0F0D0E0202804C4C0E0C4B228C053
:10155800F012133CD0F0D5F0EB02138C1218A4143F
:10156800295314A35813FA4C13F64214A74F14AF77
:0F1578004414AF49140F4314B5551499461499F0
:101587004514994716555013FE2D14022E14252B7A
:10159700140623142320163E2A13BE480000141DE8
:1015A7003F3F3F00790AA2D5202A14302C09B910F1
:1015B700020404B9080104A2D5202D025001042019
:1015C70029689229B53C005034C0E07F20302A19A1
:1015D7007F30A229722D722C500F121604C229C215
:1015E7002DC22CC22F7F30800F302C03E9C0E012B0
:1015F7001353302C03D0E0F9D0E0B53CCC302C1796
:101607007F30B9100C1213537F58302B077F788027
:1016170003B908031213533029057F2D0213537F93
:1016270020202FF87F2B202DF322922980CF286EA0
:10163700756C6C2900D2281213183028F8C2287844
:101647003C30D50108F60213BE2D504349581213FA
:10165700182403B405004001E49016509312134474
:0D166700743A121344D22A753C040214A3F5
:101ACE008B2F8A308931E4F53BF53AF539F538F547
:101ADE0036F537E533453445326012EBC0E0EAC0E7
:101AEE00E0E9C0E0AB32AA33A934121855AB2F058A
:101AFE0031E531AA307002053014F9121674F53C36
:101B0E00C394094007E53CD3940D40E1E53C6420C5
:101B1E0060DBE53CB42D054337038016E53CB42B62
:101B2E0005433701800C74FF2531F53174FF3530D4
:101B3E00F530E53560046410703FAB2FAA30A93143
:101B4E0012167464306009E535702E75350A8029D9
:101B5E0090000112168DFF64786004EFB4581343A1
:101B6E00370175351074022531F531E43530F53015
:101B7E008007E5357003753508AB2F0531E531AAC1
:101B8E00307002053014F9121674F53CC39461409E
:101B9E000AE53CD3947A5003533CDF74D0253CF5D0
:101BAE003CC3940A400CE53C9411406D74F9253CFD
:101BBE00F53CE53CD395355060433701853B408578
:101BCE003A3F85393E85383DAF357E00E4FCFDABAE
:101BDE003BAA3AA939A8381217F6C8ECC8C9EDC9FC
:101BEE00CAEECACBEFCBE4FCFDFEEB253CF53BEE9B
:101BFE003AF53AED39F539EC38F538AF3BAE3AAD4A
:101C0E0039FCAB40AA3FA93EA83DD312179650030C
:101C1E00021B87433704021B87E53720E003E4806D
:101C2E002DE53345344532601EAB2FE53124FFF9E7
:101C3E00E53034FFFAEBC0E0EAC0E0E9C0E0AB32D9
:101C4E00AA33A934121855E53730E20774FFFFFEA8
:101C5E00FDFC22E537AF3BAE3AAD39AC3830E1038F
:041C6E0002178822AF
:1017E400BB010689828A83F0225002F722BBFE01E4
:0217F400F322DE
:1017F600E88FF0A4CC8BF0A42CFCE98EF0A42CFC92
:101806008AF0EDA42CFCEA8EF0A4CDA8F08BF0A40F
:101816002DCC3825F0FDE98FF0A42CCD35F0FCEB6E
:101826008EF0A4FEA9F0EB8FF0A4CFC5F02ECD3933
:0F183600FEE43CFCEAA42DCE35F0FDE43CFC22A0
:10184500FAE6FB0808E6F925F0F618E6CA3AF622A4
:10185500BB011A89828A83D0F0D0E0F8D0E0F9D0B4
:10186500E0FAD0E0FBE8C0E0C0F00218D35016E97A
:10187500F8D083D082D0E0F9D0E0FAD0E0FBC08286
:10188500C0830218CABBFE16E9F8D083D082D0E027
:0F189500F9D0E0FAD0E0FBC082C0830218DC2259
:1018A400D083D082F8E4937012740193700DA3A3D3
:1018B40093F8740193F5828883E4737402936860E7
:0618C400EFA3A3A380DFE7
:0918CA00EBF608EAF608E9F62243
:0918D300EBF0A3EAF0A3E9F02216
:0918DC00EBF208EAF208E9F2223D
:00000001FF
